:020000020000FC
:0200000009C035
:10001400002401E0102E0FE50DBF04E00EBFC59AC9
:100024001ED000E00FBB00E00EBB01B70DBB04E027
:100034000CBB06E00CBB0000E199FECF18E0C69AA9
:10004400BE9A00E426B325FFFDCF38B3302726B38C
:1000540025FDFDCF38BB1A95A9F70000FFCF662711
:1000640050E8650F61BF000000002BD0403039F12B
:100074005695552331F0052F413009F40195600F51
:10008400F1CF413009F051E05FEF650F61BF00002F
:10009400000017D0403099F0650F61BF00000000E8
:1000A40010D0403061F05195550F550F650F61BF69
:1000B4000000000006D0403011F0BE9ACFCF462F8A
:1000C4000895332401E0402E06E202BE11E0B59B00
:1000D400FECFB599FECF13BF28B720FF02C0310C65
:1000E40048BEB59BFECF28B720FF02C0310C48BEE6
:1000F400B599FECF28B720FF02C0310C48BEB59B8E
:10010400FECF28B720FF02C0310C48BEB599FECF00
:100114000A9581F728B720FF02C0310C48BEB59B71
:10012400FECF28B720FF02C0310C48BEB599FECFE0
:1001340003BE28B720FF04C00894301C217028BFD8
:1001440022B619E526E2211632063CF41BE925E223
:100154001215230524F440E0089541E008954FEF7B
:020164000895FC
:00000001FF
